
 SYSTEM

 Start     Length     Name                   Class
 0001:0000 0044BH     _TEXT                  CODE
 0002:0000 00069H     _DATA                  DATA

 Origin   Group
 0002:0   DGROUP

 Address   Export                  Alias

 0001:018F A20_Proc                A20_Proc
 0001:0336 CreateSystemTimer       CreateSystemTimer
 0001:0319 DisableSystemTimers     DisableSystemTimers
 0001:02E0 EnableSystemTimers      EnableSystemTimers
 0001:016C Get80x87SaveSize        Get80x87SaveSize
 0001:02D3 GetSystemMsecCount      GetSystemMsecCount
 0001:0002 InquireSystem           InquireSystem
 0001:03EA KillSystemTimer         KillSystemTimer
 0001:0183 Restore80x87State       Restore80x87State
 0001:0177 Save80x87State          Save80x87State
 0001:0195 WEP                     WEP

  Address         Publics by Name

 0001:018F       A20_Proc
 0000:0000  Imp  ALLOCCSALIAS         (KERNEL.170)
 0002:000D       COPROCFLAG
 0001:0336       CreateSystemTimer
 0001:0319       DisableSystemTimers
 0002:0013       DOSVER
 0001:02E0       EnableSystemTimers
 0002:000B       FBOOTDRIVE
 0001:016C       Get80x87SaveSize
 0001:02D3       GetSystemMsecCount
 0002:000F       HIMEM
 0001:01E4       INITSYSTEM
 0001:0002       InquireSystem
 0001:03EA       KillSystemTimer
 0001:0000       MYCSDS
 0000:0000  Imp  NOHOOKDOSCALL        (KERNEL.101)
 0002:000A       NUMFLOPPIES
 0002:000C       ONEDRIVEFLAG
 0001:0183       Restore80x87State
 0001:0177       Save80x87State
 0002:0000       SYSTEMISINITED
 0001:0284       TI1
 0002:0018       TIMERTABLE
 0001:0238       TIMER_INT
 0001:0195       WEP
 0000:0000  Imp  WOW16CALL            (KERNEL.500)
 0000:0000  Imp  __0040h              (KERNEL.193)
 0000:0000  Imp  __MOD_COMMDLG        (KERNEL.532)
 0000:0000  Imp  __MOD_DGDI           (KERNEL.525)
 0000:0000  Imp  __MOD_DKERNEL        (KERNEL.521)
 0000:0000  Imp  __MOD_DUSER          (KERNEL.523)
 0000:0000  Imp  __MOD_GDI            (KERNEL.524)
 0000:0000  Imp  __MOD_KERNEL         (KERNEL.520)
 0000:0000  Imp  __MOD_KEYBOARD       (KERNEL.526)
 0000:0000  Imp  __MOD_MMEDIA         (KERNEL.531)
 0000:0000  Imp  __MOD_SHELL          (KERNEL.528)
 0000:0000  Imp  __MOD_SOUND          (KERNEL.527)
 0000:0000  Imp  __MOD_TOOLHELP       (KERNEL.530)
 0000:0000  Imp  __MOD_USER           (KERNEL.522)
 0000:0000  Imp  __MOD_WINSOCK        (KERNEL.529)
 0000:0000  Imp  __ROMBIOS            (KERNEL.173)

  Address         Publics by Value

 0000:0000  Imp  __MOD_DUSER          (KERNEL.523)
 0000:0000  Imp  __MOD_MMEDIA         (KERNEL.531)
 0000:0000  Imp  __MOD_COMMDLG        (KERNEL.532)
 0000:0000  Imp  __MOD_SHELL          (KERNEL.528)
 0000:0000  Imp  __MOD_USER           (KERNEL.522)
 0000:0000  Imp  __0040h              (KERNEL.193)
 0000:0000  Imp  ALLOCCSALIAS         (KERNEL.170)
 0000:0000  Imp  __MOD_WINSOCK        (KERNEL.529)
 0000:0000  Imp  __MOD_GDI            (KERNEL.524)
 0000:0000  Imp  __MOD_DGDI           (KERNEL.525)
 0000:0000  Imp  __MOD_KERNEL         (KERNEL.520)
 0000:0000  Imp  __ROMBIOS            (KERNEL.173)
 0000:0000  Imp  __MOD_KEYBOARD       (KERNEL.526)
 0000:0000  Imp  __MOD_TOOLHELP       (KERNEL.530)
 0000:0000  Imp  __MOD_DKERNEL        (KERNEL.521)
 0000:0000  Imp  NOHOOKDOSCALL        (KERNEL.101)
 0000:0000  Imp  __MOD_SOUND          (KERNEL.527)
 0000:0000  Imp  WOW16CALL            (KERNEL.500)
 0001:0000       MYCSDS
 0001:0002       InquireSystem
 0001:016C       Get80x87SaveSize
 0001:0177       Save80x87State
 0001:0183       Restore80x87State
 0001:018F       A20_Proc
 0001:0195       WEP
 0001:01E4       INITSYSTEM
 0001:0238       TIMER_INT
 0001:0284       TI1
 0001:02D3       GetSystemMsecCount
 0001:02E0       EnableSystemTimers
 0001:0319       DisableSystemTimers
 0001:0336       CreateSystemTimer
 0001:03EA       KillSystemTimer
 0002:0000       SYSTEMISINITED
 0002:000A       NUMFLOPPIES
 0002:000B       FBOOTDRIVE
 0002:000C       ONEDRIVEFLAG
 0002:000D       COPROCFLAG
 0002:000F       HIMEM
 0002:0013       DOSVER
 0002:0018       TIMERTABLE

Program entry point at 0001:01e4
